:100000003AC05CC05BC05AC059C058C037C156C066
:1000100055C054C053C052C051C050C04FC04EC054
:100020004DC04CC04BC04AC049C000003A00370028
:100030000000310000003B003800000032000000EA
:1000400000000000000200000001030400000000A6
:100050000404010104040404040202020202020274
:1000600002010102020104081020400102040810EC
:1000700020408004BE0211241FBECFEDCDBF10E092
:10008000A0E6B0E0EEE8F6E002C005900D92A837D9
:10009000B107D9F720E0A8E7B0E001C01D92A2396E
:1000A000B207E1F710E0CBE3D0E003C02197FE01F7
:1000B000E6D2CA33D107D1F72BD1E7C2A1CF90E066
:1000C000FC01E25CFF4F3491FC01EE59FF4F24919B
:1000D000FC01E05BFF4FE491EE23B9F0332329F0FC
:1000E0003130A1F480B78F7780BFF0E0EE0FFF1FB3
:1000F000EC5CFF4FA591B4918FB7611117C0F894D4
:10010000EC9120952E232C938FBF0895323019F453
:1001100080B78F7DE9CF333021F48FB58F778FBDD6
:10012000E4CF343011F78FB58F7DF9CFF894EC918F
:100130002E2BE9CF0F931F93CF93DF93C7E0D0E02F
:10014000082F10E0B8010C2E02C0759567950A942F
:10015000E2F7617084E0B3DF61E086E0B0DF60E089
:1001600086E0ADDF219770F7DF91CF911F910F915E
:10017000089560E085E0A3DF8FEFDCDF61E085E0DC
:100180009ECFCF93DF93C82FD62F60E085E097DF17
:100190008C2F90E0D13059F483599F4FFC0180811E
:1001A0008095C8DF61E085E0DF91CF9188CF8D59E0
:1001B0009F4FF4CF60E08230D1F0833019F181306D
:1001C00059F08AE07CDF60E089E079DF60E088E078
:1001D00076DF61E08BE073CF8BE071DF60E089E078
:1001E0006EDF60E088E06BDF61E08AE0F4CF8BE0F7
:1001F00066DF60E08AE063DF60E088E060DF61E0A6
:1002000089E0E9CF8BE05BDF60E08AE058DF60E007
:1002100089E055DF61E088E0DECFCF93DF9390E0A7
:10022000FC01EE59FF4F2491805B9F4FFC018491AC
:100230008823D1F090E0880F991FFC01E65DFF4F05
:10024000A591B491FC01EC5CFF4FC591D491623053
:1002500071F49FB7F8943C91822F809583238C93FF
:10026000E8812E2B28839FBFDF91CF9108958FB710
:10027000F894EC912E2B2C938FBFF6CF1F920F92F8
:100280000FB60F9211242F933F938F939F93AF93A9
:10029000BF9380917D0090917E00A0917F00B091EE
:1002A000800030917C0026E0230F2D3768F129E88B
:1002B000230F0396A11DB11D20937C0080937D0028
:1002C00090937E00A0937F00B0938000809178008F
:1002D00090917900A0917A00B0917B000196A11DC8
:1002E000B11D8093780090937900A0937A00B09329
:1002F0007B00BF91AF919F918F913F912F910F9074
:100300000FBE0F901F9018950296A11DB11DD4CF5E
:1003100083E080BF83BF789489B7826089BF61E042
:1003200085E07BDF61E086E078DF61E084E075DF17
:1003300061E08BE072DF61E08AE06FDF61E089E01D
:100340006CDF61E088E069DF62E080E066DF60E04A
:100350008BE0B5DE60E08AE0B2DE60E089E0AFDE2F
:1003600060E088E0ACDE809161002AE0622F3DD140
:1003700080938E0090938F0080918D0036D1809372
:1003800090009093910020E6822E2AEE922EA12CCE
:10039000B12CDAE011E08099B7C080916200813021
:1003A00091F56091610070E090E080E02CE330E036
:1003B00040E050E001D120918D00620F711D811D40
:1003C000911D28EE33E040E050E0F6D060938900C4
:1003D00070938A0080938B0090938C002FB7F894D1
:1003E00080917D0090917E00A0917F00B09180006F
:1003F0002FBF8093850090938600A0938700B093D1
:100400008800109262002FB7F89480917D0090913F
:100410007E00A0917F00B09180002FBF40918500A9
:10042000509186006091870070918800841B950B25
:10043000A60BB70BC0908900D0908A00E0908B008B
:10044000F0908C00C81AD90AEA0AFB0A1C141D0491
:100450001E041F040CF46BC010928E0010928F00CB
:1004600010929000109291002FB7F89480917D0027
:1004700090917E00A0917F00B09180002FBF4091AD
:100480008100509182006091830070918400841BF0
:10049000950BA60BB70B893C9105A105B105F0F0B2
:1004A000809161008330D0F481E0909160009111DF
:1004B00080E0809360002FB7F89480917D00909148
:1004C0007E00A0917F00B09180002FBF80938100BB
:1004D00090938200A0938300B09384008091600089
:1004E000813009F058CF8EE8E82E80E0F82EC0E089
:1004F0008C2F60DE6C2FF70181917F0142DE39DEA7
:10050000CF5FC430A9F747CF9EE8E92E90E0F92EDF
:10051000C0E08C2F4FDE6C2FF70181917F0131DE1F
:1005200028DECF5FC430A9F71093620034CFC70133
:10053000B601A501940165D0C22F20936100C701C7
:10054000B60128EE33E040E050E05BD0CA01B901CB
:100550002CE330E040E050E054D0262F60938D0033
:100560008C2F6D2F42D080938E0090938F00822F1E
:100570003CD0809390009093910076CF6091610081
:1005800070E090E080E02CE330E040E050E014D0F8
:1005900020918D00620F711D811D911D28EE33E0A9
:1005A00040E050E009D06093890070938A00809306
:1005B0008B0090938C000895EE27FF27AA27BB2776
:1005C00008C0A20FB31FE41FF51F220F331F441FE3
:1005D000551F969587957795679598F37040A9F77D
:1005E000009799F7BD01CF010895991B79E004C0E8
:1005F000991F961708F0961B881F7A95C9F7809562
:100600000895052E97FB16F400940FD057FD05D0E2
:1006100014D007FC02D046F408C0509540953095A0
:1006200021953F4F4F4F5F4F08959095809570955E
:1006300061957F4F8F4F9F4F0895A1E21A2EAA1BFD
:10064000BB1BFD010DC0AA1FBB1FEE1FFF1FA21782
:10065000B307E407F50720F0A21BB30BE40BF50B7F
:10066000661F771F881F991F1A9469F76095709508
:10067000809590959B01AC01BD01CF010895EE0FCF
:0E068000FF1F0590F491E02D0994F894FFCF30
:10068E00011E01FC60DAF266B6BEE0FEF6FD61DB2D
:08069E00F367B7BFE1FFF700AD
:00000001FF
